:100000000C94CC020C94F4020C94F4020C94F402C0
:100010000C94F4020C94F4020C94F4020C94F40288
:100020000C94F4020C94F4020C94182C0C94BB2A3B
:100030000C94F4020C94F4020C94F4020C94F40268
:100040000C94F4020C94F4020C94F4020C94F40258
:100050000C944C0C0C94F4020C94F4020C940A03CF
:100060000C94F4020C94F4020C94F4020C94F40238
:100070000C94F4020C94F4020C94F4020C94F40228
:100080000C94F4020C94F4020C94F4020C94F40218
:100090000C94F4020C94F4020C94F4020C94F40208
:1000A0000C94F4020C94F4020C94F40214001A0060
:1000B00008001500170000001C0018000C001200BA
:1000C000130004001600070009000A0000000B00DE
:1000D0000D000E000F0033001D001B00060019006C
:1000E0000500E0001100100036003700380029003C
:1000F0002B00E300E1002A00E2002C002B442D003D
:100100003400280000000000000000001E081F0846
:1001100052002F08300800004B0024002500260064
:1001200025082008500051004F00210800004E0013
:100130002100220023002E082F0030002608270867
:100140002408E00035001E001F002000310002449A
:100150004900E300E1002A00E2002C00FFFF370025
:1001600027002E00000000000000000049004A00A7
:1001700052004D004B000000520040004100420080
:1001800043004C00500051004F004E000000510051
:100190003D003E003F0044000000E9480000000030
:1001A0000060FFFF00003A003B003C0045000000FB
:1001B000EA48FFFFFFFFFFFFFFFFFFFF0160460070
:1001C0004700CD480000000000000000302E313113
:1001D0002E302B32370076657273696F6E0076654C
:1001E0007273696F6E0005010906A101050719E028
:1001F00029E715002501750195088102950175080B
:1002000081019505750105081901290591029501DE
:100210007503910195067508150025FF050719005E
:1002200029FF8100C0050C0901A1018504150026E4
:10023000FF0319002AFF03950475108100C0050112
:100240000906A1018508050719E029E71500250120
:10025000750195088102050819012908950875019D
:1002600091020507750495018101190429DD150026
:100270002501750195D98102750395018101C0059C
:10028000010980A1018505150026FF00190029FF3D
:10029000950175088100C074726967676572006DA9
:1002A0006170006D6163726F732E006D6163726FB8
:1002B000732E6D61700A6D6163726F732E74726953
:1002C000676765720044796E616D69634D61637241
:1002D0006F73004D6163726F7300656570726F6D4F
:1002E0002E657261736500656570726F6D2E667242
:1002F000656500656570726F6D2E636F6E74656EF7
:10030000747300656570726F6D2E636F6E74656EC9
:1003100074730A656570726F6D2E667265650A6525
:100320006570726F6D2E6572617365002F00637268
:10033000630076657273696F6E0076616C69643F05
:100340000064656661756C744C61796572007365F3
:100350007474696E67732E0073657474696E677365
:100360002E64656661756C744C617965720A73659B
:100370007474696E67732E76616C69643F0A736585
:100380007474696E67732E76657273696F6E0A7323
:10039000657474696E67732E63726300637573743A
:1003A0006F6D0064656661756C74006F6E6C794387
:1003B0007573746F6D006B65796D61702E006B6580
:1003C000796D61702E637573746F6D0A6B65796DED
:1003D00061702E64656661756C740A6B65796D6118
:1003E000702E6F6E6C79437573746F6D0045455058
:1003F000524F4D4B65796D61700065736361706537
:100400005F6F6E6573686F742E63616E63656C5F9A
:100410006B6579006573636170655F6F6E657368A6
:100420006F742E63616E63656C5F6B6579004573F5
:10043000636170654F6E6553686F740066616C73BD
:1004400065007472756500706C7567696E73006421
:1004500065766963652E72657365740068656C7096
:100460000A6465766963652E72657365740A706CDB
:100470007567696E730068656C70000D0A2E004D1B
:100480006F7573654B657973004F6E6553686F7454
:100490000051756B657973005370616365436164E6
:1004A000657400080B00020202000009040000014C
:1004B00002020000052400100105240101010424AA
:1004C0000206052406000107058103100040090407
:1004D0000100020A000000070502024000000705B3
:1004E000830240000012010002EF0201400912E500
:1004F000A1000101020301546563686E6F6D616EB6
:100500006379004174726575730004030904050181
:100510000902A10185010509190129081500250114
:1005200095087501810205010930093109381581E5
:10053000257F750895038106050C0A38021581256B
:100540007F750895018106C005010902A101050911
:100550001901290815002501950875018102050179
:100560000930093116000026FF7F751095028102BF
:1005700009381581257F750895018106C0001D0C7D
:10058000EB0D840E780FD70F7715B1190E231825B0
:100590002626C02C9B2E6F2F11241FBECFEFDAE032
:1005A000DEBFCDBF11E0A0E0B1E0ECEAF0E602C0B2
:1005B00005900D92A63AB107D9F724E0A6EAB1E07A
:1005C00001C01D92AA3EB207E1F712E0CCECD2E0E6
:1005D00004C02197FE010E94BE2FCF3BD107C9F76F
:1005E0000E94F7020C9454300C94000008950E946D
:1005F000C9030E94F6028AE394E00E94902C0E94B4
:100600005B05C0E0D0E00E9472052097E1F30E94F4
:100610000000F9CF1F920F920FB60F9211242F9363
:100620003F938F939F93AF93BF938091A701909136
:10063000A801A091A901B091AA013091A60123E0DF
:10064000230F2D3758F50196A11DB11D2093A6014A
:100650008093A7019093A801A093A901B093AA0148
:100660008091AB019091AC01A091AD01B091AE0130
:100670000196A11DB11D8093AB019093AC01A09395
:10068000AD01B093AE01BF91AF919F918F913F911A
:100690002F910F900FBE0F901F90189526E8230FF3
:1006A0000296A11DB11DD2CF2FB7F8946091A7017A
:1006B0007091A8018091A9019091AA012FBF08957E
:1006C0003FB7F8948091AB019091AC01A091AD013E
:1006D000B091AE0126B5A89B05C02F3F19F0019639
:1006E000A11DB11D3FBFBA2FA92F982F8827BC018C
:1006F000CD01620F711D811D911D42E0660F771FB4
:10070000881F991F4A95D1F708958F929F92AF92B3
:10071000BF92CF92DF92EF92FF926B017C010E9419
:1007200060034B015C01C114D104E104F104E9F060
:100730000E94BF2C0E946003681979098A099B09ED
:10074000683E73408105910570F321E0C21AD1081B
:10075000E108F10888EE880E83E0981EA11CB11C08
:10076000C114D104E104F10429F7FF90EF90DF9068
:10077000CF90BF90AF909F908F9008958230910559
:1007800038F0880F991F880F991F05970197F1F787
:100790000895789484B5826084BD84B5816084BDF9
:1007A00085B5826085BD85B5816085BDEEE6F0E0EA
:1007B000808181608083E1E8F0E010828081826046
:1007C0008083808181608083E0E8F0E080818160C7
:1007D0008083E1E9F0E080818260808380818160B4
:1007E0008083E0E9F0E0808181608083E1ECF0E0EB
:1007F0008081846080838081826080838081816049
:100800008083E3ECF0E0808181608083E0ECF0E0C5
:10081000808182608083E2ECF0E08081816080836F
:10082000EAE7F0E080818460808380818260808359
:1008300080818160808380818068808308950895AD
:1008400086E0ECE4F1E0DB0101900D928A95E1F79E
:1008500086E0089589E393E00E941F178CE193E0FE
:100860000E94481386E793E00E94CF1F8CEA93E032
:100870000E94832382E191E00E945C1E81E693E066
:100880000E94211A8EE393E00E94CC1887ED92E03B
:100890000E94831180E008958FE293E00E94721419
:1008A00089E393E00E94151781E693E00E94361ACF
:1008B0008EE393E00E948C1880E008958FE293E02D
:1008C0000E946F1580E00895CF93DF93EC01BC0187
:1008D00086E793E00E945F22811107C0BE018CEA87
:1008E00093E0DF91CF910C94A024DF91CF910895F4
:1008F000CF93DF93EC01BC0185E091E00E943519B4
:1009000081111CC0BE018CE193E00E941013811183
:1009100015C0BE0182E191E00E94121F81110EC03C
:10092000BE0181E693E00E94AC1A811107C0BE01AE
:1009300087ED92E0DF91CF910C946011DF91CF9120
:100940000895BC0181E693E00C94661A0F931F93FF
:10095000CF938C01BC0189E393E00E94C117C82F9B
:1009600081114BC0B80180E493E00E947619C82F32
:10097000811143C0B8018DE293E00E948D15C82F0C
:1009800081113BC0B8018EE293E00E941D16C82F72
:10099000811133C0B8018EE393E00E94E118C82FA3
:1009A00081112BC0B80187ED92E00E94B111C82FD0
:1009B000811123C04EED51E0B80180E493E00E9424
:1009C000611981111AC066ED71E0C8010E94FF2F04
:1009D000892B99F46CEC71E08DED93E00E94262751
:1009E00084E690E00E94BE0360E28DED93E00E94F9
:1009F0004A2784E690E00E94BE038C2FCF911F917E
:100A00000F91089580E00895CF93DF93EC01BC012E
:100A10008DE193E00E942614811107C0BE018DE193
:100A200093E0DF91CF910C942614DF91CF9108953C
:100A3000CF93DF93EC01BC0182E191E00E94001FA3
:100A4000BE0181E693E00E94681B80E0DF91CF91B8
:100A5000089580E493E00E94B41986E793E00E9431
:100A6000D0228CEA93E00E943E2482E191E00E9431
:100A7000711E81E693E00E94201B80E00895882388
:100A800029F08130A1F090E080E0089587E797E7B2
:100A9000909301088093000888E19BE00FB6F894DA
:100AA000A895809360000FBE90936000FFCF80E018
:100AB0000E942D0BE8CF80915301909154010E9428
:100AC000190A85E00E943F1781E08093AC0360E043
:100AD00071E087ED92E00E949811809133038F7747
:100AE0000C942D0B80915301909154010C94CC0ADD
:100AF00081E492E00E94D40D80E892E00E946E0FA3
:100B000082E692E00E94820E88EC92E00C94BB0F89
:100B1000E5E5F1E050E040E070E060E00000919138
:100B2000A92FB0E084E0B595A7958A95E1F7909656
:100B30002C9130E09F7002C0359527959A95E2F789
:100B40002095309521703327042E02C0220F331FC9
:100B50000A94E2F7622B732B4F5F5F4F4C305105C5
:100B6000E9F6CB0108951F93CF93DF93C1E1D2E063
:100B700010E0288139818A819B81482F440F42707F
:100B8000522F5170452B09F005C1AC015695479580
:100B9000440F427021FB552750F9452B09F0EFC057
:100BA000AC015695479556954795440F427022FBE8
:100BB000552750F9452B09F0D7C0AC0156954795FC
:100BC0005695479556954795440F427023FB5527F8
:100BD00050F9452B09F0BDC0AC01529542954F70BC
:100BE00045275F704527440F427024FB552750F975
:100BF000452B09F0A3C0AC015695479552954295F7
:100C00004F7045275F704527440F427025FB5527DD
:100C100050F9452B09F087C0AC010024440F551F43
:100C2000001C440F551F001C452F502D440F4270CF
:100C300026FB552750F9452B09F06AC0AC01440F3B
:100C4000452F441F550B5195440F427027FB222717
:100C500020F9422B09F052C0492F440F4270232F34
:100C60002170422B09F040C031FB222720F9492F87
:100C70004270422B79F5492F4695427032FB22276C
:100C800020F9422BE9F4292F26952695227033FB73
:100C9000442740F9422B59F4998388832A96145F9C
:100CA000103309F066CFDF91CF911F9108956BE06B
:100CB000610F80E090E00E94200C8A819B81ECCF44
:100CC0006AE0610F80E090E00E94200C39818A8107
:100CD0009B81D9CF69E0610F80E090E00E94200CF9
:100CE00039818A819B81C7CF68E0610F80E090E005
:100CF0000E94200C39818A819B81B6CF67E0610F09
:100D000080E090E00E94200C39818A819B81A4CFF1
:100D100066E0610F80E090E00E94200C288139811C
:100D20008A819B818BCF65E0610F80E090E00E941B
:100D3000200C288139818A819B816ECF64E0610F0C
:100D400080E090E00E94200C288139818A819B817B
:100D500052CF63E0610F80E090E00E94200C288178
:100D600039818A819B8138CF62E0610F80E090E019
:100D70000E94200C288139818A819B811ECF61E0ED
:100D8000610F80E090E00E94200C288139818A81E7
:100D90009B8106CF612F80E090E00E94200C28818B
:100DA00039818A819B81F1CE81E492E00E942F0DEE
:100DB000811104C081E492E00C94320D80E892E04D
:100DC0000E94B40E82E692E00C945C0E81E492E004
:100DD0000E942F0D811104C081E492E00C94CD0D8E
:100DE00080E892E00E94680F82E692E00C94490E3F
:100DF000CF93C82F81E492E00E942F0D6C2F8111B8
:100E000005C081E492E0CF910C94950D80E892E0CA
:100E1000CF910C943F0FCF93C82F81E492E00E94B2
:100E20002F0D6C2F811105C081E492E0CF910C94BD
:100E30006E0D80E892E0CF910C94180FCF93C82FDD
:100E400083FF03C081EE0E940B07C0FF03C080EE4A
:100E50000E940B07C1FF03C082EE0E940B07C2FF76
:100E600003C086EE0E940B07C4FF04C083EECF913F
:100E70000C940B07CF910895CF93C82F892F0E9410
:100E80001E078C2FCF910C940B07FC019081DB0186
:100E90008C91981305C081E0218111969C912913B2
:100EA00080E008951F93CF93DF9300D000D0CDB79B
:100EB000DEB7182F803368F5E82FF0E0EE0FFF1F44
:100EC000EB5BFB4F808191819C838B838FEF8983C8
:100ED0008A83BE016F5F7F4FCE0103960E94450754
:100EE000882369F0A12FB0E0AB54BE4FE09102011E
:100EF000F0910301612F8C9109958B839C838B81E9
:100F00009C810F900F900F900F90DF91CF911F91C8
:100F100008951092A5041092A604E5EAF4E0D2CF59
:100F20001F93CF93DF93C62F172F862F972F0E94E3
:100F3000A104823009F1812F807C61F480E28C0F62
:100F4000883008F010E08C2F912FDF91CF911F9106
:100F50000C943C07812F887C883471F4612F70E0F9
:100F6000762F66276C0F711D737082E692E0DF9119
:100F7000CF911F910C94340EDF91CF911F91089562
:100F80008F929F92BF92CF92DF92EF92FF920F9338
:100F90001F93CF93DF9300D000D000D0CDB7DEB742
:100FA0007C016B010E94E60610E000E0BB24BA94CD
:100FB0000033110599F1F6019081901729F1003362
:100FC00030F5F801EE0FFF1FEB5BFB4F8080918047
:100FD0009E828D82BB82BC82BE016D5F7F4FCE013F
:100FE00005960E94450781110FC019821A82BE0121
:100FF0006F5F7F4FCE0105960E944507811104C0A7
:10100000B401C7010E9490070F5F1F4FD1CF10920C
:10101000A5041092A604E5EAF4E0D8CF26960FB610
:10102000F894DEBF0FBECDBFDF91CF911F910F911E
:10103000FF90EF90DF90CF90BF909F908F9008959A
:10104000EF92FF920F931F93CF93DF938C01EB01ED
:10105000898181FF43C080FD41C08B81807CF1F597
:10106000888180930101FA8081E492E00E942F0D33
:101070006F2D81112EC081E492E00E94DE0D882345
:1010800001F1FB80EA80F3FE03C081EE0E94F806C6
:10109000F0FE03C080EE0E94F806F1FE03C082EE6F
:1010A0000E94F806F2FE03C086EE0E94F806F4FEE7
:1010B00003C083EE0E94F8068E2D0E94F8060E945F
:1010C000D4068B81882379F00E941E070E94D406E3
:1010D0000AC080E892E00E94020FD1CFE0910101A6
:1010E0008881E81317C0898181FF07C080FD05C092
:1010F0006A817B81C8010E949007CE010E9404058D
:101100008230E9F0DF91CF911F910F91FF90EF9026
:101110000C94D406E03360F4F0E0EE0FFF1FEB5BBD
:10112000FB4F8181982F907CF1F60E941E07DBCF48
:101130001092A5041092A604E5EAF4E0F2CFDF9144
:10114000CF911F910F91FF90EF900895FF920F9311
:101150001F93CF93DF93CDB7DEB72D970FB6F894DB
:10116000DEBF0FBECDBF8C0129873A874B875C87D6
:101170006D87203348F430FF61C031FD5FC0898541
:101180000E9452079C878B87CE0109960E947804A3
:10119000823009F447C0E985E03368F49A85F0E0CD
:1011A000EE0FFF1FEB5BFB4F90FF55C091FD53C04F
:1011B0009FEF90839183811135C01F821886BE01F5
:1011C000695F7F4FCE010B960E94450781112AC0AF
:1011D0001D821E82BE016B5F7F4FCE010B960E9467
:1011E000450781111FC0FF24FA94FB82FC82BE01D7
:1011F0006D5F7F4FCE010B960E944507811112C093
:10120000F982FA82BE016F5F7F4FCE010B960E947A
:101210004507811107C08C85843409F5CE010996F4
:101220000E94BE0B2D960FB6F894DEBF0FBECDBF49
:10123000DF91CF911F910F91FF9008958FEF8983D8
:101240008A83BE016F5F7F4FCE010B960E944507D8
:10125000811195CF99CF9C852B852083ABCF8F7C37
:101260008134B9F48A851B8581FF0AC080FD08C0DE
:10127000612F88EC92E00E94BF0F10930902D2CF39
:10128000809109028113CECF88EC92E00E94BD0FBD
:10129000C9CFBE01675F7F4FC8010E94C007BE0172
:1012A000675F7F4FC8010E942008CE0109960E9407
:1012B0001805B8CFEF92FF920F931F93CF93DF9350
:1012C00000D000D000D01F92CDB7DEB7022F2B8305
:1012D0003C834D835E836F83203308F042C07C01E2
:1012E000832F817031FF22C081113BC08FEF898332
:1012F0008A83BE016F5F7F4FCE0105960E9445072E
:10130000882329F0802F0E9452079E838D83CE016F
:1013100003960E946404811124C02B813C814D817D
:101320005E816F81C7010E94A6081BC08823C9F097
:1013300010E0000F111F0B5B1B4FF80180819181A2
:101340009E838D8319821A82BE016F5F7F4FCE010B
:1013500005960E9445078823D1F28FEFF80180831C
:10136000818327960FB6F894DEBF0FBECDBFDF9105
:10137000CF911F910F91FF90EF900895CF930FB6EB
:10138000F894A89580916000886180936000109225
:1013900060000FBEA5E5B1E041E651E061E070E01C
:1013A0008D91E82FF0E024E0F595E7952A95E1F797
:1013B000C1A18F709B0101C0220F8A95EAF7922F7D
:1013C00090959C2391A382A1822B82A34A175B074D
:1013D00039F7A1E6B1E045E651E061E070E08D91BA
:1013E000E82FF0E094E0F595E7959A95E1F791A163
:1013F0008F709B0101C0220F8A95EAF7922B91A36F
:1014000082A1822B82A34A175B0749F780E1809370
:1014100081001092800080EE9EE29093870080937E
:10142000860081E18093810081E080936F00CF91FD
:1014300008950E9478058CE092E00E94BE0940E881
:1014400055E260E070E08DED93E00E9420260E945E
:101450001F040E944C04E5E4F4E081E39FEF815017
:1014600021F0908391833296FACF84EB91E00C9433
:101470002B0B6F927F928F929F92AF92BF92CF92DF
:10148000DF92EF92FF920F931F93CF93DF9321E6AA
:10149000E22E21E0F22EC1E1D2E035E6632E31E00A
:1014A000732E912C812CAA24A394B12CF701819145
:1014B0007F01082F10E0159507951595079515954F
:1014C000079515950795F80192A18F70650101C0E8
:1014D000CC0C8A95EAF7892F8C2582A30E94880577
:1014E000F80122A1C226C2A24885598584279527E2
:1014F0006C817D812E813F81262737272823392340
:101500003F832E83FB01E095F095E823F923FD83CB
:10151000EC838623972320953095822393234827B5
:10152000592759874887882A992A8114910401F1FB
:101530008091190290911A029093140280931302E1
:10154000809123029091240290931E0280931D02A9
:1015500080912D0290912E02909328028093270271
:101560008091370290913802909332028093310239
:101570002A966E147F0409F099CFDF91CF911F91C5
:101580000F91FF90EF90DF90CF90BF90AF909F9022
:101590008F907F906F9008950E9454036093B001E4
:1015A0007093B1018093B2019093B3010E945E04E5
:1015B00080910C02882331F010920C028CE092E0B2
:1015C0000E94390A0E94B3050C94290570E090E34B
:1015D000899F600D711D1124660F771FFB01E45573
:1015E000FF4F8491FB01E355FF4F94910895EF92D3
:1015F000FF920F931F93CF93DF93E5EBF1E080E32E
:10160000DF011D928A95E9F77F0110E01033E1F0C8
:10161000C0910401D0E0CB51DE4FB1E0C53EDB0705
:1016200071F00A91E0910201F0910301612F802F86
:1016300009958F3F11F49F3F81F3F70100831F5FEE
:10164000FFEFEF1AFF0AE2CFDF91CF911F910F91C9
:10165000FF90EF9008950C94F70A9091000189177C
:1016600008F080E091E0909304018093E5010E94EE
:10167000F70A0C9402054091040150E090E0682FB5
:1016800070E0292F092E000C330B2417350764F462
:101690002B513E4FF9012081022E000C330B2617EF
:1016A000370721F09F5FEDCF80E0089581E0089536
:1016B000CF93909100018917A0F4C82F0E943B0B93
:1016C00081110FC0E091040181E08E0F809304012D
:1016D000F0E0EB51FE4FC0830E94F70ACF910C94CB
:1016E0000205CF910895CF93DF93D82F0E943B0B33
:1016F000882381F1C0910401C23028F480E0DF9199
:10170000CF910C942D0BE5EEF1E090E080E02D2FD1
:1017100030E04191042E000C550BBC016F5F7F4FF0
:101720004217530799F44C2F50E0481B590B6B514B
:101730007E4F8B519E4F0E942C30C150C0930401AC
:101740000E94F70ADF91CF910C940205CB016C1730
:1017500000F3F6CFDF91CF910895E0910401F0E01E
:10176000EC51FE4F80818F5F0C94580BE091040187
:10177000F0E0EC51FE4F80810C94730BCF93DF931C
:10178000FC01C2819181292F2270C43558F0222397
:1017900009F450C090FD4EC08CEA8C0FDF91CF91C0
:1017A0000C942D0BCA32C8F1D6EDDC0FD13251F0BA
:1017B000D23281F4222351F090FD08C0DF91CF9105
:1017C0000C94AD0B2223D1F390FDF8CFDF91CF9194
:1017D0000C94B60B211110C0A5E4B4E081E3815054
:1017E000B9F09C91C91306C011962C911197938161
:1017F000291701F11296F3CF90FDEECF8D2F0E94A5
:101800003B0B811117C08D2FDF91CF910C94580B9A
:101810008D2FDF91CF910C94730B222359F090FD03
:1018200009C08C2F0E943B0B882311F08C2FF1CF25
:101830008C2FEACFDF91CF9108951092090208957D
:10184000CF93DF9300D000D01F92CDB7DEB7262F05
:10185000342F842F817041FF15C0811115C08091F4
:10186000440461E0680F609344044FEF5FEF8FEA38
:1018700091E00F900F900F900F900F90DF91CF910C
:101880000C945A098111EBCF0F900F900F900F908D
:101890000F90DF91CF9108951F920F920FB60F9284
:1018A00011248F9381E080930C028F910F900FBED3
:1018B0000F901F901895FC0182818F5BFB01808344
:1018C00081E00895CF93DF93CDB7DEB769970FB668
:1018D000F894DEBF0FBECDBFFC01DB019C919F5F82
:1018E0009C939E012D5F3F4F81E1D9011D928A9506
:1018F000E9F729E0298384E08A8391E09D8383E0EE
:101900008E839F8398872A8721E22B879C879D87D8
:101910009F8722E2288B2FE3298B27E02B8B25E062
:101920002C8B8E8B20E430E0388F2F8B998F828127
:101930008B83838180688D8B49E150E0BE016F5FAE
:101940007F4F80E00E946A2A69960FB6F894DEBF46
:101950000FBECDBFDF91CF910895FC01DB018C91CB
:101960008138A9F413968C911397823281F42281E5
:1019700014968D919C912817190649F48285848FBD
:101980004FE350E066EE71E080E80C946A2A90E044
:1019900080E00895FC01DB01228114968D919C91D9
:1019A00015972817190681F511968C9111979C911E
:1019B000913A69F4813029F0833029F4848D809341
:1019C000F10081E008958230F9F4858DF8CF9132ED
:1019D000D9F48B3021F412968C91848FF2CF8A3017
:1019E00011F4158EEECF893079F4CF0116962D9132
:1019F0003C91179713964C91423041F461E070E0AE
:101A00004E962130310551F080E008954130E1F7E4
:101A100028303105C9F768E070E00B960E94902AE3
:101A2000D0CFCF93DF93EC0181E08C838D839E0137
:101A3000255E3F4F3F832E831986188629E631E0C5
:101A4000398328836A876C8F8D8F1E8E81EC8B8FF4
:101A50000E940327BE01DF91CF910C94BF26FC01A9
:101A6000848D0895EF92FF920F931F93CF93DF938E
:101A70008C01EC012B967C0183E1E80EF11C48E01F
:101A800050E0BE01C7010E941630892B21F1F801F8
:101A9000838148E050E0BE0180640E94B9298C0136
:101AA000E0916002F0916102309731F09C0148E0D2
:101AB00050E0BE0182E0099588E0FE01D701019067
:101AC0000D928A95E1F7C801DF91CF911F910F9197
:101AD000FF90EF9008950FEF1FEFF5CFFC0180E22C
:101AE000860F883070F4605E770B21E030E001C033
:101AF000220F6A95EAF78385822B838781E090E045
:101B00000895DF011D9690E080E02D912617B1F336
:101B1000211104C0E80FF91F6587F0CF01968630C8
:101B2000910599F790E080E00895CF93DF9320E24C
:101B3000260F283090F4605E770B21E030E001C082
:101B4000220F6A95EAF72095FC013385232323872A
:101B500081E090E0DF91CF910895DC011D969C011A
:101B60002D5E3F4FFD014191461303C0EF012197C8
:101B70001882E217F307B9F720E03D91332349F0CB
:101B8000EC01C20FD11D4D853D87ED0121974883A2
:101B90002F5FAE17BF0789F7DBCF0B9628E0FC015C
:101BA00011922A95E9F70895CF93DF93EC010E94F3
:101BB000CD0DCE01DF91CF910C94320DFC013D96FD
:101BC00043962191261729F0E817F907D1F780E00D
:101BD000089581E008952091390230913A024091B0
:101BE0003B0250913C0260913D0270913E02809117
:101BF0003F0290914002A1E00E94DE2F2093390223
:101C000030933A0240933B0250933C0260933D0272
:101C100070933E0280933F02909340020E94EA2F0D
:101C200029F461E081E492E00C94110D0895809113
:101C30007202811113C010927B0210927A0285E227
:101C400092E090937D0280937C0289E190E09093F2
:101C50007F0280937E0281E0809372020E94272E91
:101C60006AE772E00C94942DFC0130E020E0419191
:101C70005191452B41F4220F331F280F391FF901D1
:101C80007183608308952F5F3F4F2430310579F7CA
:101C9000089528E0FC0111922A95E9F70895CF9361
:101CA000DF93EC010E94272E28E030E0AE0164E0D3
:101CB000DF91CF910C94E42D0F931F93CF93DF937B
:101CC000EC018C01085F1F4F48E050E0BC01C801E7
:101CD0000E941630892B51F0CE010E944F0E88E0F1
:101CE000FE01D80101900D928A95E1F7DF91CF9125
:101CF0001F910F91089528E0FC0111922A95E9F7B0
:101D00000C945C0E0C947B0E82E692E00C94170E01
:101D10008091BA02811113C01092C3021092C202C4
:101D20008EE392E09093C5028093C40281E490E038
:101D30009093C7028093C60281E08093BA020E940A
:101D4000272E62EC72E00C94942DCF93DF93EC017C
:101D50000E94272EAE01435E5F4F2DE130E068E028
:101D6000DF91CF910C94E42DEF92FF920F931F938C
:101D7000CF93DF93EC01F8808D8D8E010F5F1F4FA5
:101D80008F15D9F0F801AE01435E5F4F20E0858DDD
:101D900030813196932F9095982319F08323848F67
:101DA00021E0E417F50799F7222319F0CE010E94EC
:101DB000A50EFD8ECE010E94A50E7E018EE1E80EDD
:101DC000F11C4CE150E0B801C7010E941630892B8C
:101DD00081F08CE1F801D70101900D928A95E1F72D
:101DE000CE01DF91CF911F910F91FF90EF900C9456
:101DF000A50E8FEF9FEFDF91CF911F910F91FF9075
:101E0000EF9008956E3D90F4E62FE695E695E69501
:101E1000E80FF92FF11D677021E030E001C0220FBB
:101E20006A95EAF79181922381E009F480E00895B0
:101E30006E3DA0F4E62FE695E695E695E80FF92FBE
:101E4000F11D677021E030E001C0220F6A95EAF7CA
:101E50008181822B818381E090E00895605E68300B
:101E600058F441E050E001C0440F6A95EAF7FC01E4
:101E70002081242B2083EFCF90E080E008956E3DF9
:101E8000A8F4E62FE695E695E695E80FF92FF11D03
:101E9000677021E030E001C0220F6A95EAF72095D3
:101EA00081812823218381E090E00895605E68307D
:101EB00060F421E030E001C0220F6A95EAF7209536
:101EC000FC01308123232083EECF90E080E0089551
:101ED0002DE1FC0111922A95E9F70895CF93DF9344
:101EE000EC010E94680FCE01DF91CF910C94A50EFA
:101EF00080E892E00C94880E8091C902811113C091
:101F00001092D2021092D1028FE792E09093D40205
:101F10008093D30288E190E09093D6028093D5021B
:101F200081E08093C9020E94272E61ED72E00C943B
:101F3000942D0F931F93CF93DF93EB018A010E949F
:101F4000272E9801AE0165E0DF91CF911F910F918F
:101F50000C94E42DCF93DF931F92CDB7DEB7198297
:101F600041E050E0BE016F5F7F4F0E94990F0F90DC
:101F7000DF91CF9108950C94AA0F0C94AA0FCF93E0
:101F8000DF931F92CDB7DEB76983633841F48AE3EC
:101F900094E00E94A32C0F90DF91CF91089541E02F
:101FA00050E0BE016F5F7F4F0E94990FF4CF88EC25
:101FB00092E00C947C0F0C943E308F929F92AF92E3
:101FC000BF92CF92DF92EF92FF920F931F93CF9326
:101FD000DF938C01FC01E080F18015821482C280C5
:101FE000D380CE0CDF1C4701B12C8C149D0408F06B
:101FF0004BC0E4012196C4010E94DB0F8E3008F033
:1020000043C0E82FF0E0E95FFF4E0C94BE2F36107E
:10201000151015101910191019101510151015108C
:102020001710171017101C102B10E40122964E01E8
:10203000DCCFE4012396FBCF4E01CE010E94DB0FE3
:10204000A82E2296C40101960E94DB0FA110F4CFA6
:102050008111F2CFECCF2C2F9D2F2196822F0E9441
:10206000DB0F2C2F9D2F8111F8CFE1CFB394EB2DF7
:10207000F0E03296EE0FFF1FE00FF11FCE018E1938
:102080009F0991838083D3CF8B2DDF91CF911F91B7
:102090000F91FF90EF90DF90CF90BF90AF909F9007
:1020A0008F9008958F929F92AF92BF92CF92DF92BE
:1020B000EF92FF920F931F93CF93DF93FC01EC5BA2
:1020C000FF4F2081621708F0DFC07C01E62FF0E0AF
:1020D0003296EE0FFF1FEE0DFF1DD7010D911C91E3
:1020E00080819181080F191FD12CF7018081918186
:1020F00022813381820F931F0817190708F0C4C08B
:10210000E8012196C8010E94DB0F81508D3008F054
:10211000BBC0E82FF0E0E157FF4E0C94BE2FBB1080
:10212000CA10D610E710F810091115112111C210AC
:10213000C210C2109C102D118D2C912CB12CA12CF1
:10214000CE010E94DB0FC82E8E010E5F1F4FCE0105
:1021500001960E94DB0F811102C0CC2091F0682F04
:102160007C2D8DE193E00E940114C501B4010E9411
:102170008503E801E5CF0E5F1F4FCE010E94DB0F04
:10218000D82EE8016D2D70E090E080E00E9485037C
:102190008E01ABCF0E5F1F4FCE010E94DB0F682F69
:1021A00070E090E080E00E948503EBCFCE010E94BA
:1021B000DB0FC82EE8012396C80102960E94DB0FB0
:1021C000682F7C2D8DE193E00E945D13DBCFCE0163
:1021D0000E94DB0FC82EE8012396C80102960E94D8
:1021E000DB0F682F7C2D8DE193E00E949813CACFFE
:1021F000CE010E94DB0FC82EE8012396C80102968B
:102200000E94DB0F682F7C2D8DE193E00E9401146A
:10221000B9CF0E5F1F4FCE010E94DB0F682F70E019
:102220008DE193E00E945D13ACCF0E5F1F4FCE0196
:102230000E94DB0F682F70E08DE193E00E949813FD
:10224000A0CF0E5F1F4FCE010E94DB0F682F70E002
:102250008DE193E00E94011494CFCE018D2C912C3E
:10226000B12CA12C21960E94DB0F882309F48ACF80
:10227000682F70E08DE193E00E940114C501B40164
:102280000E948503CE01EECFDF91CF911F910F9178
:10229000FF90EF90DF90CF90BF90AF909F908F9086
:1022A0000895292F30E0322F222790E08C55914D50
:1022B000280F391F81E02032310508F080E00895B1
:1022C0000F931F93CF93DF938C01EB018A819B8146
:1022D0000E9451118823A9F0898181FF0DC080FDE2
:1022E0000BC06A816C55C8010E94521081E0DF91D9
:1022F000CF911F910F9108958DE193E00E94C0133B
:10230000F5CF80E0F4CF65EC72E08DED93E00E94B4
:10231000262784E690E00E94BE036AE08DED93E0FC
:102320000E944A2784E690E00E94BE0380E0089560
:102330000F931F93CF93DF93EC018B018FE293E018
:102340000E94C014998388831B830A83CE010E9454
:10235000DD0FCC5BDF4F8883DF91CF911F910F9111
:102360000895BF92CF92DF92EF92FF920F931F9347
:10237000CF93DF93EC018B014BEA52E080E493E0D2
:102380000E946119811186C047E050E063EA72E063
:10239000C8010E940830892B09F07CC0095F1F4FDB
:1023A0006FE972E0C8010E94FF2F892B09F05FC01E
:1023B0008DED93E00E943225F12CE12C8A309105BD
:1023C00011F0019621F58A819B81E816F90608F043
:1023D0004EC0888199818E0D9F1D0E94DB0F4AE0BF
:1023E00050E0682F8DED93E00E94C02784E690E0D6
:1023F0000E94BE0360E28DED93E00E944A2784E6CE
:1024000090E00E94BE038FEFE81AF80ADCCF8DED52
:1024100093E00E9432258A30910511F1019601F175
:102420008A819B81E816F906D8F441E070E060E00B
:102430008DED93E00E943528B62E67018FEFC81A04
:10244000D80A88819981E80EF91EC7010E943E30A2
:10245000B81621F06B2DC7010E9446307601D7CF08
:10246000CE010E94DD0FFE01EC5BFF4F808367E928
:1024700072E0C8010E94FF2F892B51F441E070E007
:1024800060E08DED93E00E943528CE010E9452104D
:1024900081E001C080E0DF91CF911F910F91FF900B
:1024A000EF90DF90CF90BF9008958F929F92AF9260
:1024B000BF92FF920F931F93CF93DF93EB0120976F
:1024C00009F4A4C0F12C8E010F5F1F4FFE0184910F
:1024D000EFEFE80FED3008F099C0F0E0EE58FD4E58
:1024E0000C94BE2FAF12BB12C412D112DE12EB122B
:1024F000F412FD12B312B312B3127F129A128F2C80
:10250000912CB12CA12CB801F80184916F5F7F4F01
:102510000E5F1F4FFB016491611102C0882319F106
:10252000782F8DE193E00E940114C501B4010E944F
:102530008503E9CF8F2C912CB12CA12C0F5F1F4F5D
:10254000F80131976491662371F070E08DE193E0BA
:102550000E940114C501B4010E948503EFCF2296A9
:10256000F801F4908E016F2D70E090E080E00E9401
:102570008503E801A8CF2296F801649170E090E00D
:1025800080E00E948503EECFF80174918E010D5F0B
:102590001F4FFE01329664918DE193E00E945D131E
:1025A000E2CFF80174918E010D5F1F4FFE0132964C
:1025B00064918DE193E00E949813D5CFF801749156
:1025C0008E010D5F1F4FFE01329664918DE193E005
:1025D0000E940114C8CF2296F801649170E08DE149
:1025E00093E00E945D13BECF2296F801649170E0E3
:1025F0008DE193E00E949813B5CF2296F801649183
:1026000070E08DE193E00E940114ACCFDF91CF9197
:102610001F910F91FF90BF90AF909F908F90089562
:102620000F931F93CF93DF93EB012B8130E0322F79
:1026300022274A8150E0BA017056260F371F2F3FDC
:10264000310509F0F8F48C01BE01842F0E943F058A
:10265000BC01C8010E945512898180FF02C081FF20
:102660000DC08A8190E090562B8130E0322F2227D6
:10267000820F931F8F3F910529F020F08DE193E0A9
:102680000E94C01380E0DF91CF911F910F910895B8
:1026900063ED72E08DED93E00E94262784E690E0E2
:1026A0000E94BE036AE08DED93E00E944A2784E613
:1026B00090E00E94BE0380E00895EF92FF920F9396
:1026C0001F93CF93DF9300D000D01F92CDB7DEB71A
:1026D0008C01F62EE72E609144048FEF898382E807
:1026E0008A83FB827C836D832FEF32E84F2D572F37
:1026F0008FEA91E00E94A608C8014096F801E81709
:10270000F90741F02081211111C0218121110EC052
:10271000F082E1820F900F900F900F900F90DF9159
:10272000CF911F910F91FF90EF9008953296E7CFD0
:10273000CF93DF9300D000D01F92CDB7DEB7AB01AF
:102740009C01205F3F4FFC012E173F0751F0808115
:10275000841305C08181851302C0108211823296D4
:10276000F3CF609144042FEF31E88FEA91E00F90AE
:102770000F900F900F900F90DF91CF910C94A608BF
:10278000CF92DF92EF92FF920F931F93CF93DF933D
:1027900000D000D01F92CDB7DEB77C0120E1E20E61
:1027A000F11C8C01DD24DA9481E8C82EE016F106D4
:1027B000D1F0F80140815181411102C0552381F0CF
:1027C00060914404D982CA824B835C836D832FEF6E
:1027D00031E88FEA91E00E94A608F8011082118288
:1027E0000E5F1F4FE3CF0F900F900F900F900F9041
:1027F000DF91CF911F910F91FF90EF90DF90CF90DD
:1028000008950F931F93CF93DF9300D000D01F92B2
:10281000CDB7DEB78B01609144042FEF32E8A801F9
:102820008FEA91E00E94A608609144042FEF31E8FE
:10283000A8018FEA91E00F900F900F900F900F90EA
:10284000DF91CF911F910F910C94A6080F931F93C6
:10285000CF93DF938C01005F1F4FEC010C171D0716
:1028600071F06881798189819881911102C08823F2
:1028700021F08FEA91E00E9490072296EFCF80E04E
:10288000DF91CF911F910F91089584E690E00C9411
:10289000BE034AE050E0682F8DED93E00E94C02710
:1028A0000E94451460E28DED93E00E944A270C944B
:1028B0004514FF920F931F93CF93DF93EC01F62EF5
:1028C00008811981C8010E943E30F81621F06F2D51
:1028D000C8010E944630CE01DF91CF911F910F9128
:1028E000FF900895AF92BF92CF92DF92EF92FF9246
:1028F0000F931F93CF93DF9300D0CDB7DEB78C013A
:102900006C0184E0C80ED11C5601F12CE12CC701EA
:102910000E943E30F50181935F01FFEFEF1AFF0A3D
:1029200084E0E816F10499F7F80185818F3FD1F42E
:102930008481982F9F779F3711F487FD148281E05F
:10294000F801858310E000E01A830983F6016191A4
:102950006F01CE0101960E9459140F5F1F4F043082
:10296000110591F780E00F900F90DF91CF911F91AB
:102970000F91FF90EF90DF90CF90BF90AF900895B0
:102980000F931F93CF93DF9300D0CDB7DEB77A8339
:102990006983FC01238110E000E021110FC0008158
:1029A0001181CB01800F911F9183808342E0BE0192
:1029B0006F5F7F4F87E393E00E94BD16C8010F90C1
:1029C0000F90DF91CF911F910F910895CF92DF92D9
:1029D000EF92FF920F931F93CF93DF9300D0CDB769
:1029E000DEB77C016C0184E0C80ED11C10E000E071
:1029F0001A830983F60161916F01CE0101960E944D
:102A000059140F5F1F4F0430110591F781E0F70152
:102A100082830F900F90DF91CF911F910F91FF90C4
:102A2000EF90DF90CF9008951F93CF93DF93EC0149
:102A3000162F80910001681748F4862F0E942D0BF5
:102A40008C818078912F9F77892B8C831E3720F083
:102A50008C8180788E678C83CE010E94E6148C81F5
:102A60008F77DF91CF911F910895FC01948160FBD6
:102A700097F99483892F8F778F3719F490789E6711
:102A80009483CF010C94E614CF93DF93EC0181E0A3
:102A90008B8360E187E393E00E94A4168D818130EF
:102AA00021F01A82DF91CF9108952E813F8180918C
:102AB0003703909138032F3F320769F49F838E8349
:102AC000CE010E94E6148C818F778E3758F7DF9104
:102AD000CF910C942D0B2817390721F7F4CFFC0167
:102AE0002381211102C00E94441580E0089584E0F2
:102AF00090E09093300380932F0308958DED93E041
:102B00000E9432259C0181E02A30310529F02F3FB7
:102B10003F4F11F080E0089508950F931F93CF93D6
:102B2000DF9300D0CDB7DEB78B0143E053E080E404
:102B300093E00E946119811133C063EF72E0C80114
:102B40000E94FF2F892BF1F40E947E1510E000E017
:102B5000811147C00E947E1581113BC041E070E0A9
:102B600060E08DED93E00E9435281A830983CE0141
:102B700001960E9459140F5F1F4F011584E018073A
:102B800049F727C067EE72E0C8010E94FF2F892B2A
:102B900049F06AED72E0C8010E94FF2F892B69F1AC
:102BA00080E018C080912F039091300360E074E0C2
:102BB000681B790B4AE050E08DED93E00E94C72737
:102BC0000E94451460E28DED93E00E944A270E9426
:102BD000451481E00F900F90DF91CF911F910F91DD
:102BE0000895C8010E943E300E9449140F5F1F4F94
:102BF000011584E01807A9F7ECCF10E000E01A8374
:102C000009836FEFCE0101960E9459140F5F1F4F89
:102C1000011584E0180799F787E797E79093010873
:102C20008093000888E19BE00FB6F894A895809304
:102C300060000FBE90936000FFCFCF93DF93EB0156
:102C400048E553E080E493E00E94611981117AC065
:102C500049E050E06EE473E0CE010E940830892B19
:102C600009F070C0299661E473E0CE010E94FF2F45
:102C7000892B81F40E947E15811160C041E070E0D3
:102C800060E08DED93E00E9435288FE293E00E9492
:102C9000141540C06AE373E0CE010E94FF2F892B18
:102CA000E9F162E373E0CE010E94FF2F892B71F1FD
:102CB0006EE273E0CE010E94FF2F892B09F042C023
:102CC00080913203D0E0C0E0882321F0C091350329
:102CD000D091360360913703709138034AE050E099
:102CE0008DED93E00E94C7270E9445146CE273E0CB
:102CF0008DED93E00E9426270E9445144AE050E0A3
:102D0000BE018DED93E00E94C72715C0809134036A
:102D10000E94491481E0DF91CF91089560913103C1
:102D200080E493E00E94A6190E94451460E28DEDB4
:102D300093E00E944A270E944514ECCF8091330310
:102D40008F77E6CF80E0E7CFFC01208131812170D1
:102D5000332781E0861770F440815181569547955D
:102D600051834083220F331F41705527242B352B6D
:102D70008F5FF0CF318320830895DC01FB01415048
:102D800000F181912D913C91119768E070E051E044
:102D9000982F952399F4932F991F9927991F220F04
:102DA000331F992319F095E029273058550F6150AA
:102DB000710971F711963C932E93E1CF932F909563
:102DC000EBCF089584E690E00C94BE031F93CF935D
:102DD000DF9390913B03891730F080E090E0DF9122
:102DE000CF911F910895C62FD0E090E3899FC00D29
:102DF000D11D1124CC0FDD1F60913C0370913D0368
:102E0000C60FD71FCE010E943E30182FCE0101966B
:102E10000E943E30912FE3CF90913A03891710F42E
:102E20000C94E60A891B0C94E6168FE293E00E944C
:102E300072148091000180933A0380E008956DEE52
:102E400073E08DED93E00E9426270E94E2166AE06F
:102E50008DED93E00E944A270E94E21680E00895DB
:102E600080933B0390E6899FB00111248FE293E0A9
:102E70000E94C01490933D0380933C030895809377
:102E800000019091330326EE36E197FD07C0909143
:102E90003A03980F909300012CE037E1309303013F
:102EA000209302010C943017FF920F931F93CF933E
:102EB000DF9300D0CDB7DEB7F62E672F8C01000F61
:102EC000111F80913C0390913D03800F911F9A83C5
:102ED0008983CE0101960E94591480913C03909100
:102EE0003D030196800F911F9A8389836F2DCE0138
:102EF00001960E9459140F900F90DF91CF911F916E
:102F00000F91FF900895FF920F931F93CF93DF933C
:102F1000F82E8B01C0E0CF15F9F0D0E06D2F8C2F8B
:102F2000F8010995692F70E0762F6627680F711DEB
:102F30004AE050E08DED93E00E94C7270E94E21620
:102F400060E28DED93E00E944A270E94E216DF5F67
:102F5000D03321F7CF5FDFCFDF91CF911F910F915A
:102F6000FF9008958DED93E00E9432259C0181E051
:102F70002A30310529F02F3F3F4F11F080E00895AE
:102F80000895FF920F931F93CF93DF931F92CDB7B6
:102F9000DEB78B014EEB53E080E493E00E946119B1
:102FA00081118EC047E050E066EB73E0C8010E94DB
:102FB0000830892B09F084C0095F1F4F6BEA73E06A
:102FC000C8010E94FF2F892BE1F50E94B2178823C8
:102FD000B1F06091330367FB662760F94AE050E087
:102FE0008DED93E00E94C0270E94E21660E28DED15
:102FF00093E00E944A270E94E21681E062C041E00D
:1030000070E060E08DED93E00E943528162F698313
:103010008FE293E00E94351590913B03909300015D
:10302000112339F086EE96E190930301809302011B
:10303000E4CF80913A03890F809300018CE097E1FF
:10304000F3CF63EA73E0C8010E94FF2F892B39F4A4
:1030500066EE7AE080913A030E948317CECF6CE946
:1030600073E0C8010E94FF2F892B51F50E94B2170F
:1030700010E000E090E3F92E882329F066EE76E177
:1030800080913B03E9CF0E94B2178111B6CF8091A6
:103090003B038F9DC00111240817190708F0ADCF1D
:1030A00041E070E060E08DED93E00E943528272F2D
:1030B0003327722FC8010E9454170F5F1F4FE3CFB1
:1030C00080E00F90DF91CF911F910F91FF900895B5
:1030D000FF920F931F93CF93DF93EC018B01FB01C2
:1030E000F0800E943E30F81621F06F2DCE010E9434
:1030F0004630F801F1802196CE010E943E30F8164C
:1031000021F06F2DCE010E944630C801DF91CF9192
:103110001F910F91FF900895CF92DF92EF92FF924F
:103120000F931F93CF93DF937C0162E070E08FE2F7
:1031300093E00E94C014EC01F701918380838C011D
:103140006C01F2E0CF0ED11C0C151D0540F4C80136
:103150000E943E308F3F41F40F5F1F4FF5CF65E077
:1031600071E0CE010E946818F701C081D181CE01C3
:103170000E943E3080930501CE0101960E943E30B0
:103180008093060180E0DF91CF911F910F91FF9016
:10319000EF90DF90CF9008956EE274E08DED93E0B4
:1031A0000E94262784E690E00E94BE036AE08DED2F
:1031B00093E00E944A2784E690E00E94BE0380E0EC
:1031C00008950F931F93CF93DF93EC018B0144E19C
:1031D00054E080E493E00E946119811144C06AEFD9
:1031E00073E0C8010E94FF2F892BE9F58DED93E074
:1031F0000E9432258A309105C9F00196B9F041E06C
:1032000070E060E08DED93E00E9435286093050149
:103210007093060165E071E0888199810E946818C9
:1032200081E0DF91CF911F910F9108956091060188
:1032300070E0762F662780910501680F711D4AE0C6
:1032400050E08DED93E00E94C72784E690E00E9455
:10325000BE0360E28DED93E00E944A2784E690E091
:103260000E94BE03D7CF80E0DCCFCF93DF93DC0199
:10327000EB019A818C91981305C02B8111968C914A
:10328000281749F09E3721F080E0DF91CF91089513
:103290008B81813DC9F7898181FFF6CF80FDF4CF15
:1032A00087FDF2CF82E191E00E946A1D882361F3DD
:1032B00061E082E191E00E94CE1D1A821B8281E0D2
:1032C000E4CFCF93DF93CB01EA0166E774E00E947D
:1032D000FF2F892B49F4BE018DED93E00E94552705
:1032E00081E0DF91CF91089580E0FBCFCF93DF9312
:1032F000EB014CE554E00E946119811125C06FE497
:1033000074E0CE010E94FF2F892B89F487E797E7AD
:10331000909301088093000888E19BE00FB6F89431
:10332000A895809360000FBE90936000FFCF67E484
:1033300074E0CE010E94FF2F892B31F40E942A04F1
:1033400081E0DF91CF91089580E0FBCF611106C04D
:103350006CE374E08DED93E00C94262762E474E056
:10336000F9CF109260030895CF93DF93EC018DEDB8
:1033700093E00E9448258DED93E00E944B25892B18
:1033800009F45BC08DED93E00E945B25E8A191E01C
:103390009E0F98A3EC0FFD2FF11D8083FE01E90F16
:1033A000F11D31978081803271F0903260F48DEDA3
:1033B00093E00E944B25892B31F08DED93E00E9424
:1033C00032250A97F9F68881811107C018A280E298
:1033D000FE0111928A95E9F730C0E8A1EC0FFD2FAC
:1033E000F11D319780818032F9F4E8A1E150FF0BA3
:1033F000EC0FFD1F8081803209F41082CE010E9403
:10340000A6048DED93E00E944B25892B31F08DEDC4
:1034100093E00E945B258A30A1F76BE774E08DEDA5
:1034200093E00E945527D2CF8DED93E00E94322584
:103430000A97D9F288A18032C0F680E0DF91CF915F
:1034400008956FE774E08DED93E00E94262784E6EF
:1034500090E00E94BE036AE08DED93E00E944A274F
:1034600084E690E00E94BE0380E00895CF93DF934E
:1034700000D000D000D0CDB7DEB782EC94E00E943F
:10348000992EE6EDF4E0108A8685978524853585AA
:1034900019823B832A839D838C831E820284F38559
:1034A000E02D0190F081E02D46E050E0BE016F5F1D
:1034B0007F4F80EE94E0099580E026960FB6F89451
:1034C000DEBF0FBECDBFDF91CF910895FC017035F7
:1034D00079F4862F8076803429F49085862F8F7B2F
:1034E000892B8087862F807729F48781682B6783D3
:1034F00080E008958031E1F780E1689FB0011124F8
:10350000F4CFCF93DF93EC0182EC94E00E945C2E29
:10351000688582EC94E00E94622E82EC94E0DF9158
:10352000CF910C94742EFB01928196FB222720F9F7
:1035300080E090FD82E0822B20E091FD24E0822B50
:1035400020E092FD28E0822B93FD04C090E0892BBF
:103550000C94DE1B90E1FBCFFB012381203559F455
:10356000DC0117961C9217972281322F3076303467
:1035700021F418961C9280E0089525FFFCCF21814C
:1035800021FFF9CF20FDF7CF0E94931AF4CF2091AD
:10359000B0013091B101FC01318320839681892FE4
:1035A0008F7019F410926C03089580910F0181952A
:1035B00092FF80E093FF03C020910F01820F609182
:1035C0000F01619590FF60E091FF03C090910F01A2
:1035D000690F0E94801C82EC94E00C94742E0F936F
:1035E0002091B0013091B101FC01358324838681A3
:1035F00090E024E0959587952A95E1F70097F1F002
:1036000000910901019582FF00E083FF03C0209132
:103610000901020F2091090180FF20E081FF03C012
:1036200080910901281B40E060E082EC94E00E9458
:10363000542E82EC94E00F910C94742E0F91089507
:10364000CF93DF93EC018091B0019091B1012A8179
:103650003B81AC01421B530B9A0140910A015091EE
:103660000B012417350780F09B838A8320916C031C
:1036700030910C014FEF50E0431B51092417150600
:103680001CF4230F20936C0328813981821B930B38
:1036900020910D0130910E018217930718F0CE0191
:1036A0000E94C71A8091B0019091B1012C813D8197
:1036B000821B930B20910701309108018217930719
:1036C00018F0CE010E94EF1A80E0DF91CF910895AB
:1036D0000F931F93CF93DF93FB0123812035C9F410
:1036E0008B01EC0182818076803419F4CE010E9436
:1036F000811A8F818E831F82F8018281807779F40D
:103700008091B0019091B1019B838A83CE010E9488
:10371000C71A80E0DF91CF911F910F9108958031FA
:10372000C1F7CE010E94EF1AF4CFCF93DF9300D000
:1037300000D000D0CDB7DEB736952795820F931F06
:1037400056954795640F751FE6EDF4E095878487DD
:1037500077876687208929839B838A837D836C830F
:103760001E820284F385E02D0190F081E02D46E079
:1037700050E0BE016F5F7F4F80EE94E00995269682
:103780000FB6F894DEBF0FBECDBFDF91CF91089585
:1037900010926F0310926E031092710310927003D7
:1037A0008FEF9FE790937503809374039093730357
:1037B0008093720381E080936D0308950F931F93AC
:1037C000CF93C82F80916D03811102C00E94C81B46
:1037D000C0FF06C010926D03CF911F910F91089505
:1037E000E09111010E2F10E0809174039091750308
:1037F000B8010E94742F9B0170937503609374034A
:103800008091720390917303B8010E94742FAB01F1
:1038100070937303609372036C2F6470E091700374
:10382000F091710380916E0390916F037C2F7670FD
:10383000763091F4820F931F90936F0380936E0301
:10384000BA016E0F7F1F7093710360937003CF9165
:103850001F910F910C94951B662349F1D801119784
:10386000A49FB001A59F700DB49F700D1124E60FA9
:10387000F71FF0937103E0937003C4FF1DC0015064
:103880001109029FB001039F700D129F700D11244A
:10389000860F971F90936F0380936E036091700360
:1038A0007091710380916E0390916F03D0CFC1FD31
:1038B000E4CFE40FF51FDDCFC3FDF0CF820F931FE0
:1038C000E9CF482F50E087FD0AC0889FC00111242E
:1038D000880F892F881F990B91958F5F089520E09D
:1038E00031E0241B350B229FC001239F900D900DCA
:1038F0001124880F892F881F990B91958095089521
:10390000EF92FF920F931F93CF93DF93082F162F01
:10391000C0911001D0E0F12CE12C8823D1F08091EE
:103920006C030E94611C20916B03382F0303C001BC
:103930001124820F911D27FD9A957E01C817D90782
:1039400044F0EE24FF24EC1AFD0AE816F9060CF404
:103950007C01112309F449C080916C030E94611C11
:1039600020916A03382F1303C0011124820F911D87
:1039700027FD9A95C817D9073CF0D195C195D10973
:10398000C817D9070CF4EC0110926D03AE01D7FFF4
:1039900002C0415F5F4F94E0559547959A95E1F7D6
:1039A000B701F7FE02C0615F7F4F84E075956795B0
:1039B0008A95E1F700E020E082EC94E00E94542E2A
:1039C00020E130E0C701B9010E94882F80936B038A
:1039D000CE01B9010E94882F80936A03DF91CF91B5
:1039E0001F910F91FF90EF900895D0E0C0E0CCCFF1
:1039F000FC018281DB019C91891730F5A081B181A6
:103A0000A80FB11D2C9130E0938102C03595279508
:103A10009A95E2F724834481442391F0242F30E0E7
:103A2000938140FF07C0880F880F880F890F858317
:103A300081E008953595279524839F5F9383EBCF8D
:103A40008F5F82831382D5CF80E00895262F26953D
:103A500026952695820F911DFC01808190E067706C
:103A600002C0959587956A95E2F781700895E62FD3
:103A7000E695E695E695E80FF92FF11D677081E070
:103A800090E0A0E0B0E004C0880F991FAA1FBB1F00
:103A90006A95D2F72081822B80830895E62FE695E0
:103AA000E695E695E80FF92FF11D862F877041E026
:103AB00050E060E070E004C0440F551F661F771FA0
:103AC0008A95D2F7409550956095709580814823EE
:103AD00040830895EF92FF920F931F93CF93DF934C
:103AE000CDB7DEB72C970FB6F894DEBF0FBECDBFB3
:103AF0008C010A9698878F8319861A86FF24FA9478
:103B0000FC869A83898386E0E82EEB821C82FE8203
:103B1000BE016D5F7F4FCE0107960E94F81C811198
:103B200013C0005F1F4F18870F8319861A86FC8603
:103B30001A830983EB821C82FE82BE016D5F7F4F78
:103B4000CE0107960E94F81C2C960FB6F894DEBFA3
:103B50000FBECDBFDF91CF911F910F91FF90EF90DE
:103B60000895272F207C69F4605E683098F4FC018A
:103B70008681978102C0969587956A95E2F7817054
:103B80000895743439F426ED260F2A3218F462525F
:103B9000603168F381E008950C94B11DAF92BF923B
:103BA000DF92EF92FF920F931F93CF93DF93CDB7E6
:103BB000DEB761970FB6F894DEBF0FBECDBF8C01A4
:103BC0000A967C01662381F1580190E1A90EB11C8F
:103BD000B886AF8219861A868FEF8C87BA82A9823F
:103BE00096E09B831C828E83BE016D5F7F4FCE016A
:103BF00007960E94F81C8823B9F0DC846D2DC5015E
:103C00000E944E1D6D2DC7010E944E1D60914404FF
:103C10002D2D31E84FEF5FEF8FEA91E00E94A6086B
:103C20008A858F5F8A87E0CFF886EF8219861A86A9
:103C30008FEF8C87FA82E98296E09B831C828E83C9
:103C4000005F1F4FBE016D5F7F4FCE0107960E9440
:103C5000F81C882309F1DC846D2DC8010E94261D03
:103C60006D2D8823A9F0C8010E944E1D6D2DC7013E
:103C70000E944E1D609144042D2D31E84FEF5FEFFF
:103C80008FEA91E00E94A6088A858F5F8A87DACF43
:103C9000C7010E944E1DF8CF61960FB6F894DEBFA3
:103CA0000FBECDBFDF91CF911F910F91FF90EF908D
:103CB000DF90BF90AF90089569E874E08DED93E0D8
:103CC0000E94262784E690E00E94BE036AE08DED04
:103CD00093E00E944A2784E690E00E94BE0380E0C1
:103CE00008954F925F926F927F928F929F92AF92C0
:103CF000BF92CF92DF92EF92FF920F931F93CF93D9
:103D0000DF93CDB7DEB761970FB6F894DEBF0FBE75
:103D1000CDBF8C01FC0160807180C090B001D0905B
:103D2000B10186899789C81AD90A8280938078015F
:103D3000FAE0EF0EF11CF886EF8219861A868FEFF3
:103D40008C87FA82E98296E09B831C828E83512CB9
:103D5000580180E1A80EB11CBE016D5F7F4FCE01FE
:103D600007960E94F81C482E882349F15C84652D33
:103D7000C5010E94261D8823D1F0C614D70490F0F7
:103D8000652DC5010E944E1D652DC7010E944E1D67
:103D900060914404252D31E84FEF5FEF8FEA91E009
:103DA0000E94A6088A858F5F8A87542CD5CFC814B5
:103DB000D904C0F3652DC7010E944E1DF3CF5110E9
:103DC00007C08091B0019091B101F801978B868B6B
:103DD00080E061960FB6F894DEBF0FBECDBFDF91D5
:103DE000CF911F910F91FF90EF90DF90CF90BF90F8
:103DF000AF909F908F907F906F905F904F900895BD
:103E00000C94711E872F90E0982F8827860F911DA4
:103E10002FEF280F283018F4815290E008958F5D1D
:103E200094E40895AF92BF92CF92DF92EF92FF9207
:103E30000F931F93CF93DF93FB01B180B7FC5BC05F
:103E4000EB018C016C01FAE0CF0ED11C6881C60138
:103E50000E94261DA82E780180E1E80EF11C6881E1
:103E6000C7010E94261DB1FE90C0B0FC8EC0A110FB
:103E700051C0811185C08A819B81292F30E0322F6A
:103E80002227482F50E04150504C240F351F20313D
:103E9000310598F46A817B81C8010E94021F9B83CF
:103EA0008A836881C6010E94371D8091B00190917C
:103EB000B101F801978B868B1BC0F8012085222366
:103EC00039F0292F207C21F420E2280F283048F3F4
:103ED000F8012185222331F0943421F426ED280FB6
:103EE0002A32F8F2292F207C41F4805E883050F489
:103EF0008881F801808F80E038C0943419F48A52A8
:103F00008A32B0F3F8018689978920813181821B3A
:103F1000930BD0CF882361F36881C6010E944E1DA8
:103F20009881F801808D981729F06881C7010E9457
:103F30004E1DDECF6A817B81C8010E94CC1D882383
:103F4000A1F3F8018481958197FF02C0808191815E
:103F50002091B0013091B101F80146895789241BA5
:103F6000350B2817390708F782E0DF91CF911F91B1
:103F70000F91FF90EF90DF90CF90BF90AF9008959A
:103F80006881C6010E944E1DD0CFA11003C08823B6
:103F900009F4B1CF6881C7010E94371DE5CF61E9FF
:103FA00074E08DED93E00E94262784E690E00E9465
:103FB000BE036AE08DED93E00E944A2784E690E01C
:103FC0000E94BE0380E00895FC01872F90E0982FA7
:103FD0008827680F792F711D613180EC7807E0F038
:103FE000623188EC780750F46151704C66A717A6CF
:103FF00011AA80EE870F80AB81E00895633180EDD8
:10400000780750F46251784C66A717A68AE2870FAA
:1040100080AB84E481ABF0CF80E008958F929F92D3
:10402000AF92BF92CF92DF92EF92FF920F931F93C6
:10403000CF93DF9300D000D0CDB7DEB78C01F62E42
:104040002FE2261708F469C0E62FF0E0EE0FFF1FFD
:10405000EB5BFB4FD080E1808FEFD8120FC0E812EE
:104060000DC0AF2DB0E0AB54BE4FE0910201F09116
:1040700003016F2D8C910995D82EE92E6D2D7E2D83
:10408000C8010E94E41FB82E811135C0EF2DF0E069
:10409000EB54FE4F8080C12CAA24AA94912CF801E5
:1040A0008281C81608F042C0F4E0CF9EC0011124FE
:1040B000F80160817181680F791FAA8244E050E0A5
:1040C000CE0101960E94F62F89819A813B812C8135
:1040D000F9122AC0482F082E000C550B4815590517
:1040E00011F08F3F09F5F801D6A6E7A6C90190ABFC
:1040F00021ABBB24B3948B2D0F900F900F900F909A
:10410000DF91CF911F910F91FF90EF90DF90CF90B3
:10411000BF90AF909F908F9008951092A504109239
:10412000A604E5EAF4E096CFC394B9CFD6A6E7A6F5
:104130008FEF80AB81ABDFCFCF93DF93FC01EB013F
:104140009A01261B370BA4E6B0E00E94C42F26A1DB
:1041500030E050E040E00E949C2F8091B0019091AF
:10416000B101BC016C1B7D0B81E06217730708F085
:1041700080E0DF91CF910895292F207C39F490E2DF
:10418000980F81E0983048F080E007C09434E1F760
:1041900096ED980F81E09A32B8F70895CF93DF93A8
:1041A000EC018881681780F5882371F1815088833C
:1041B000E62FF0E0DF011196AC0FBD1FEE0FFF1FE1
:1041C0007196EC0FFD1F962F981780F411962C9185
:1041D00011972D9318962C91189717962C93179743
:1041E00022813381219331939F5FEECF2FEF30E017
:1041F00001C0220F6A95EAF789A1922F9095982322
:1042000086958223892B89A3DF91CF910895CF933F
:10421000DF9300D000D01F92CDB7DEB7FC0134850C
:1042200084A1982F917080FD28C082E02481398379
:104230008A836B837C832D8391110AC0872F90E042
:10424000982F8827680F792F711D64307105F0F45D
:1042500060E0CF0103960E94CE2029813A814B81F4
:104260005C816D818FEA91E00F900F900F900F901D
:104270000F90DF91CF910C945A0981E0D7CF6D3226
:10428000710530F36933710518F703C068327105A1
:10429000B0F78489958994A783A7DACFCF93DF936A
:1042A000FC017381DC011D9681E090E060E08717DE
:1042B000F0F452A94D9124A130E0082E02C03595AA
:1042C00027950A94E2F720FD0DC0541721F080E0F5
:1042D000DF91CF9108952489358934AB23AB682FC2
:1042E0000196E5CF5413FCCF8FEF82ABF0CF8091D6
:1042F000B0019091B10123A934A9821B930B25A988
:104300002817190609F068F48FEF82AB6623F9F2DB
:10431000EF012396CE010E94CE2060E0CE010E94E4
:10432000CE2081E0D5CF7F928F929F92AF92BF92A5
:10433000CF92DF92EF92FF920F931F93CF93DF9371
:10434000EC019B81911110C0F12C8F2DDF91CF9149
:104350001F910F91FF90EF90DF90CF90BF90AF90A3
:104360009F908F907F9008959C848CA180FF13C0B4
:10437000983041F460E070E0CE010E940721FF24F4
:10438000F394E3CF8AA99812F5CFCE010E944E2173
:104390008111DACFEFCF692DCE010E940E20882344
:1043A00009F470C0FDA0FF2009F46CC00EA51FA584
:1043B000C8010E94BC20882E8091B0019091B1016B
:1043C0002BA53CA5821B930B2AA52817190609F0DB
:1043D00010F57B80A090B001B090B1016E0101E0BA
:1043E00010E0E12C202F071508F065C08CA190E0AB
:1043F000002E02C0959587950A94E2F780FD12C0C1
:10440000811040C0EE2009F454C07FEFC71AD70ACC
:104410000F5F1F4FE7CF8110DCCFB801CE010E94A4
:104420000721D7CFF6019585FE013D9681E09912CF
:104430002DC0EE2019F08EA1811110C0882059F0F6
:1044400068A979A99AAA8C899D899CAB8BABCE016E
:104450000E9407217ACF6EA57FA5F4CFF801EE0F59
:10446000FF1FEC0FFD1F44895589EE2DF0E0EE0F84
:10447000FF1FEC0FFD1F64897589CE010E949C20EF
:104480008111C3CF6EA57FA577CF8F5F821708F00C
:10449000BCCF31913913F9CF4C895D89B501641BCB
:1044A000750B39A53617170609F078F768A979A9A9
:1044B000CECFE02EAACF88E0781246CFE3CF0F937D
:1044C0001F93CF93DF93EC01FB0124818DA5922FE5
:1044D000981B19162CF08B8181111CC080E025C01F
:1044E0002DA780818033D0F7818187FDF7CF8B01A5
:1044F0008DA181111FC062817381CE010E94E41FD2
:10450000882361F38EA59FA5D80113969C938E9363
:104510001297E4CF022E000C330B8C81281B31093B
:1045200087FD339537FDDACF82E0DF91CF911F9180
:104530000F9108952B81822F90E03481FE01E80FC6
:10454000F91F3483DB013C913487880F991FFE01EA
:10455000E80FF91F8091B0019091B101958B848B88
:1045600011964C913CA181E090E0A0E0B0E0022ED9
:1045700004C0880F991FAA1FBB1F0A94D2F740FFDF
:104580000CC041FD0AC0832B8CA32F5F2B83CE016F
:104590000E9493218111FBCFC7CF80958323F4CF55
:1045A0000F931F93CF93DF93EC012091B0013091D3
:1045B000B1018AA590E04BA55CA5B901641B750B00
:1045C0006817790738F0A90141505109481B590B68
:1045D0005CA74BA78B818823D9F08C899D89281BE8
:1045E000390B8FA198A52817390768F00EA51FA5CC
:1045F000C8010E94BC20B801811102C068A979A934
:10460000CE010E940721CE010E9493218111FBCF90
:1046100080E0DF91CF911F910F910895CF93DF93A9
:10462000C6E7D3E0198218821A821B8288E0E0E490
:10463000F1E0A2E8B3E001900D928A95E1F781E004
:104640008DA380E58EA38AEF90E098A78FA382E3E5
:1046500089A78BE48AA780E091E09CA78BA78FEFC6
:104660008DA78EA78FA788AB89AB8AAB88EC8DAB63
:10467000DF91CF910895FC018FEF818312824091E9
:1046800048015091490160914A0170914B01478363
:10469000508761877287848B8091C10381112CC000
:1046A00081EE8093C9031092CA0386E28093CB0304
:1046B00088E08093CC031092CE031092CD0395EE48
:1046C0009093CF031092D00397E29093D1038093FD
:1046D000D2031092D4031092D3031092D5031092F8
:1046E000D6031092D7031092D8031092DA031092D7
:1046F000D90381E08093C10389EC93E09093DC03BC
:104700008093DB03089568E974E08DED93E00E94E7
:10471000262784E690E00E94BE036AE08DED93E0D8
:104720000E944A2784E690E00E94BE0380E008953C
:1047300080E026E0E091DB03F091DC03829FE00D56
:10474000F11D1124908191110FC0318131110CC0E4
:104750003281311109C03381311106C04481558144
:10476000452B11F48FEF0895961303C0918197178D
:1047700011F08F5FDFCF08950F931F93CF93DF93D7
:10478000CDB7DEB72A970FB6F894DEBF0FBECDBF08
:104790008C01FC01838980FD48C082E0F8012781FB
:1047A00093812E838F838FEF888789879A876623EB
:1047B00021F1948997FD21C09081923079F4609124
:1047C0004404298391E09A838B838C836D8331E049
:1047D0004FEF5FEF8FEA91E00E94A608F80184890D
:1047E000E091DB03F091DC0396E08902E00DF11D1E
:1047F00011248281938199878887F8018281882397
:10480000E1F0815082833396D8011B9690E098178F
:1048100070F4218121932481238312962D913C9160
:1048200013972D933D939F5FF2CF81E0B7CFF801AF
:10483000838990E095958795838B2E813F8148856C
:1048400059856A858FEA91E02A960FB6F894DEBF03
:104850000FBECDBFDF91CF911F910F910C945A09DC
:10486000CF93DF93EC018A81882329F060E0CE01A9
:104870000E94BC23F8CFDF91CF910895FC01828183
:10488000882311F120912B0130912C018489A09172
:10489000DB03B091DC0396E08902A00DB11D112469
:1048A00014968D919C91009709F09C018091B00124
:1048B0009091B10143855485841B950B8217930712
:1048C00018F0CF010E94302480E00895CF93DF9349
:1048D000FC01EB012081822F90E03C81DF01A80FD9
:1048E000B91F11963C931197388115963C93880F08
:1048F000991FDF01A80FB91F8091B0019091B101FC
:104900001A969C938E9319979981818941E050E082
:1049100060E070E0022E04C0440F551F661F771F31
:104920000A94D2F790FF09C091FD07C0482B418B34
:104930002F5F2083DF91CF91089540954823F7CFD3
:104940000F931F93CF93DF93EC01FB018481998137
:10495000282F291B12164CF09A8191111CC080E05F
:10496000DF91CF911F910F9108958983208120338A
:10497000B0F7818187FDF3CF382F327081FF1FC0E0
:1049800080FD1DC09281983591F49381913DB9F4D9
:10499000188281E0E5CF082E000C990B2B81821B39
:1049A000910927FD939597FDDACF82E0D9CF99350C
:1049B00031F49381913D19F481E08883D1CF9881BE
:1049C000913069F28F019A81992371F080FF09C0BB
:1049D000311107C08F81821323C061E0CE010E9494
:1049E000BC23CE010E943024F801818181FFB7CF22
:1049F00080FDB5CF62817381CE010E9498238C8B9C
:104A000087FDADCF8881823069F4F8012081318142
:104A10004281538164818FEA91E00E94A60802C01E
:104A20009430F9F2B801CE0102960E946624BDCFFF
:104A30008CEA93E00C943B23CF93DF931F92CDB786
:104A4000DEB76983DC01ED91FC910280F381E02DFA
:104A500041E050E0BE016F5F7F4F09950F90DF91FD
:104A6000CF910895CF93DF93EC018C859D8597FFBF
:104A700005C082E00E9488299D878C878C859D8552
:104A8000DF91CF91089583E00E949F2990E00895DF
:104A900083E00C940E2CFC018485958597FD06C05F
:104AA00082E00E94382990E00196089582E00E94F9
:104AB000382990E00895FC018485958597FD05C00F
:104AC0002FEF3FEF35872487089582E00C948829E3
:104AD000CF93DF93EC0180913801882331F083E09C
:104AE0000E94B9291816190634F081E090E09B83E2
:104AF0008A8380E090E0DF91CF910895EEEFFFE7A9
:104B00002591349181E02B3F3C4D09F080E00895E0
:104B1000FC0190819E5F908342E450E063EA74E080
:104B200080E80C946A2AFC0181819081913A61F4B9
:104B3000813209F083C047E050E061E371E080E03A
:104B40000E946A2A81E00895913209F077C0833289
:104B500069F482819381B0E0A0E080932D0190936D
:104B60002E01A0932F01B0933001ECCF803239F4A5
:104B700067E070E081E391E00E94902AE3CF823207
:104B800009F78281809338010E947E25E0E0F8E0F9
:104B9000882311F0EEEFFAE080913101909132011B
:104BA000A0913301B0913401803B9440A105B1053F
:104BB000D9F48091380180FD17C0EE3F8AE0F807F4
:104BC00071F587E797E791838083809160008093F8
:104BD0002D0488E19BE00FB6F894A89580936000BF
:104BE0000FBE90936000AECF808191818737974749
:104BF00009F0A8CFA895809160008861809360003B
:104C000080912D0480936000EE3F8AE0F80789F0E0
:104C10008091FE0A9091FF0A9183808393CF8081D7
:104C200091818737980769F29093FF0A8093FE0A73
:104C3000C8CF1092FF0A1092FE0A84CF80E0089538
:104C40002FEF3FEFFC01358724870895EDEDF3E06A
:104C50001382128288EE93E0A0E0B0E08483958313
:104C6000A683B78385E791E0918380838FEF9FEFE1
:104C7000958784870895EF92FF920F931F93CF93A8
:104C8000DF937B01FC01C281D38110E000E020971B
:104C900091F0E881F9810280F381E02DB701CE0126
:104CA000099597FD06C0080F191F0884D985C02DE6
:104CB000EECF0FEF1FEFC801DF91CF911F910F9142
:104CC000FF90EF9008950F931F93CF93DF938B0185
:104CD000FC01C281D381209771F0E881F9810480C1
:104CE000F581E02DB801CE010995009731F40884D3
:104CF000D985C02DF0CF90E080E0DF91CF911F915A
:104D00000F9108950F931F93CF93DF938B01FC01B5
:104D1000C281D381209771F0E881F9810680F78103
:104D2000E02DB801CE010995080F111D0884D98521
:104D3000C02DF0CFF8011082DF91CF911F910F911C
:104D400008950F931F93CF93DF938B01FC01C281D2
:104D5000D381209771F0E881F9810190F081E02DF5
:104D6000B801CE010995811105C00884D985C02DEF
:104D7000F0CF80E0DF91CF911F910F910895CF93F5
:104D8000DF93FC01DB01218114968C911497820F33
:104D90009927991F08978CF5C281D381209731F507
:104DA00073836283908112969C93129713962C932F
:104DB000139715968C911597890F808380E0149630
:104DC0009C9114978917E8F41696CD91DC9117976A
:104DD000C80FD11D9881C181D0E0C75CDE4F988398
:104DE00091819F5F91838F5FEACFEC0188859985E0
:104DF0000097D9F7B987A887D5CF80E0DF91CF9109
:104E0000089581E0FBCF80912E0481110DC082E0D6
:104E10008093360484E08093370410923904109212
:104E2000380481E080932E0486E394E00895FB012A
:104E300001900020E9F73197AF01461B570BDC01C9
:104E4000ED91FC910280F381E02D0994EF92FF92A5
:104E50000F931F93CF93DF938C017B01D0E0C0E0D1
:104E6000F701EC0FFD1F6491662361F0D801ED910D
:104E7000FC910190F081E02DC8010995892B11F07A
:104E80002196EECFCE01DF91CF911F910F91FF9030
:104E9000EF900895DC01ED91FC910190F081E02DFF
:104EA000099463E871E00C9417270F931F93CF9335
:104EB000DF93EC010E9426278C01CE010E9451272E
:104EC000800F911FDF91CF911F910F9108958F92C5
:104ED0009F92AF92BF92EF92FF920F931F93CF9347
:104EE000DF93CDB7DEB7A1970FB6F894DEBF0FBE44
:104EF000CDBF7C01FA01CB0119A2223008F42AE0CF
:104F00008E010F5D1F4F822E912CB12CA12CBF0161
:104F1000A50194010E949C2FF901CA016A300CF589
:104F2000605DD8016E938D01232B242B252B79F7FF
:104F300090E080E0109721F0BD01C7010E94172783
:104F4000A1960FB6F894DEBF0FBECDBFDF91CF9113
:104F50001F910F91FF90EF90BF90AF909F908F9017
:104F60000895695CDECF2115310541F4DC01ED9136
:104F7000FC910190F081E02D642F09940C94672737
:104F80009A01462F50E070E060E00C94B3279A013C
:104F9000AB0170E060E00C94B3270F931F93CF93A5
:104FA000DF93EC010E945403688779878A879B8787
:104FB000E881F9810484F585E02DCE01099597FFFC
:104FC00015C00E945403088519852A853B85601BFE
:104FD000710B820B930B0C811D812E813F81601719
:104FE00071078207930720F38FEF9FEFDF91CF9137
:104FF0001F910F910895FF920F931F93CF93DF930B
:10500000EC018B01F42ECE010E94CD2797FD1DC02F
:105010008D329105D1F09C01205331092A303105A0
:10502000A0F0FF2019F08E32910579F001301105C2
:1050300051F00230110589F48D30910571F05CF466
:105040000997029750F08FEF9FEFDF91CF911F915B
:105050000F91FF9008958097B1F7E881F98102845C
:10506000F385E02DCE010995CECFBF92CF92DF928E
:10507000EF92FF920F931F93CF93DF938C01C42F76
:1050800040E00E94FB27FC01C12CD12C760197FD4A
:105090003EC0B12C0C2E000CDD0BCE17DF07D9F073
:1050A000ED32F10509F43FC0CF01C0970A9798F49B
:1050B000AAE0B0E0A70196010E94D32F6F01FF0F75
:1050C000EE08FF08C60ED71EE81EF91E80E3C81AB8
:1050D000D108E108F108D801ED91FC910284F38533
:1050E000E02DC8010995C8010E94CD27FC01C09799
:1050F0000A9798F2CE17DF0781F2BB2041F0F094B7
:10510000E094D094C094C11CD11CE11CF11CC701D7
:10511000B601DF91CF911F910F91FF90EF90DF903B
:10512000CF90BF900895BB24B394D5CF40913D0458
:1051300050913E0420913B0430913C0442175307A8
:10514000B4F49091E8009570E1F39091E80092FD3D
:1051500019C08093F10080913D0490913E04019626
:105160008F739927892B19F48EEF8093E800809133
:105170003D0490913E04019690933E0480933D043B
:1051800081E0089580E00895EF92FF920F931F93BE
:10519000CF93DF93F82E192FE62E042F81E0860F90
:1051A000880F0E94962883E00E949628CF2DD12F49
:1051B000EC0EFD2EF11CCE15DF05B9F007FF13C074
:1051C000FE0184910E949628182F80E00E94962864
:1051D000812321968111EFCFDF91CF911F910F9104
:1051E000FF90EF9008958881EDCF81E0F5CF809119
:1051F000D70081608093D70080EA8093D80089B57A
:10520000806189BD89B5826089BD09B400FEFDCF8A
:1052100061E070E080E090E00E9485038091D8001A
:105220008F7C80618093D8008091E000807F8093A4
:10523000E0000895CF93DF931F92CDB7DEB71982B8
:10524000CE0101960E9488250E940327BE016F5F50
:105250007F4F0E943B2689810F90DF91CF91089567
:105260002FB7FC012083F89467706093E9000895DC
:10527000CF93DF931F92CDB7DEB7682FCE01019693
:105280000E9430298091F20099819FBF0F90DF9199
:10529000CF910895EF92FF920F931F93CF93DF93D7
:1052A0001F92CDB7DEB790914104992371F157FD5C
:1052B0002CC08A017B01682FCE0101960E94302903
:1052C0008091F20090E0081719070CF4C801282F0C
:1052D000F70144E6215030F0409342043091F10050
:1052E0003193F8CF009739F02091F200211103C0DB
:1052F0002BE62093E80029812FBF0F90DF91CF91FB
:105300001F910F91FF90EF9008958FEF9FEFF5CFD2
:10531000CF93DF931F92CDB7DEB741E050E0BE01DF
:105320006F5F7F4F0E944A29019731F4898190E095
:105330000F90DF91CF9108958FEF9FEFF9CFCF932B
:10534000DF931F92CDB7DEB7682FCE0101960E9482
:1053500030299091E800892F807295FF04C09091C8
:10536000F20080E4891B99819FBF0F90DF91CF915C
:1053700008955F926F927F928F929F92AF92BF92A9
:10538000CF92DF92EF92FF920F931F93CF93DF9311
:105390001F92CDB7DEB7982E6B01B42E052F8091EA
:1053A0004104811113C08FEF9FEF0F90DF91CF91D8
:1053B0001F910F91FF90EF90DF90CF90BF90AF9033
:1053C0009F908F907F906F905F90089580913F04A1
:1053D00080FF05C08091E00082608093E000EB2CAC
:1053E000F02EA12C8AEF882E892D8072682E892DAF
:1053F0008074582E9AE3792EE114F10419F4AA204E
:1054000009F457C0892D0E949F29182F81110AC0C5
:105410008A94882041F261E070E080E090E00E9490
:105420008503EACF8E151F0411F00CF01E2D692D97
:10543000CE0101960E9430298091E80085FD03C0CD
:1054400089818FBFD9CF812F90E0E81AF90A6620B1
:1054500029F01150A0F01092F100FBCFF60197FC5B
:105460000AC0115050F021912093F100FACF2491FD
:105470002093F10031961150D0F7C80ED91EAA2002
:1054800021F07092E800A12CDBCF8091E80085FD2F
:1054900008C07092E800AA24A394E114F10481F2F8
:1054A000F2CFE114F10461F6552051F27092E80058
:1054B000C7CF84E6809343048B2D902F76CF109234
:1054C000E90010923E0410923D0490933C048093B6
:1054D0003B040895DF92EF92FF920F931F93CF93B7
:1054E000DF93D82E8A01EB017B01E40EF51ECE1569
:1054F000DF0559F0D7FE12C0FE0184910E94962864
:1055000021968111F4CF0FEF1FEFC801DF91CF91EA
:105510001F910F91FF90EF90DF9008958881EECF5B
:10552000CF93DF93EC019B01B4E6ABEF211531057E
:10553000F1F0A9012134310514F040E450E08091EC
:10554000E80082FFFCCF942FFB01E21BF30BEC0F72
:10555000FD1F915028F08091F10080833196F9CFA2
:10556000B0934204A093E800241B350BDFCFCB019E
:10557000DF91CF9108951F920F920FB60F921124D1
:10558000CF92DF92FF920F931F932F933F934F93EE
:105590005F936F937F938F939F93AF93BF93EF939B
:1055A000FF93CF93DF93CDB7DEB76C97DEBFCDBF50
:1055B0001092E9008091E80083FF2FC089E0FE018E
:1055C0007596FE2E0F2F815029F09091F100908357
:1055D0003196F9CF84E68093420482EF8093E8000D
:1055E0008D8987FF38C09091E80090FFFCCF982FFD
:1055F000907609F000C19E894F89588D2F89188DAA
:10560000911130C0803859F5809140048093F100A9
:105610001092F1008EEF8093E8006C960FB6F8942C
:10562000DEBF0FBECDBFDF91CF91FF91EF91BF9154
:10563000AF919F918F917F916F915F914F913F912A
:105640002F911F910F91FF90DF90CF900F900FBE81
:105650000F901F9018959EEF9093E800C8CF10927E
:10566000F100D6CF913059F48111D4CF413051059A
:1056700089F6809140048D7F80934004CBCF933096
:1056800049F48111C7CF4130510521F68091400482
:105690008260F2CF953041F48091E80080FFFCCF2A
:1056A00020682093E300B6CF963009F076C0CB8C0B
:1056B000DC8C123039F590E080E00E945F2A0E9475
:1056C0001A291F8299E099831A8391E09E8390EAB8
:1056D00098879AEF998720913D0430913E04275F87
:1056E0003F4F3C832B838D83C6010E945F2A49E094
:1056F00050E0BE016F5F7F4F80E00E946A2A0E94E7
:105700001A2988CFC6010E945F2A0E9403276F2DA5
:10571000702F0E946326009731F00CF07BCF81E25E
:105720008093EB007ACF113061F11330C1F78F898C
:10573000882381F1823049F440E866E083E095E017
:105740000E94C428882359F365CF813029F440E8AA
:105750006BE087EF94E0F4CF833009F70E940327D2
:105760008E010F5F1F4FB8010E948226F801019041
:105770000020E9F73197BF01601B710B40E0C801C1
:10578000DFCF65EE74E0FB01449150E080E80E94B9
:105790006A2A40CF6AE075E0F6CF973009F4BFCFB0
:1057A000983021F481E08093F10034CF993009F0F2
:1057B00031CF837009F0B3CFEAE3F1E081E031E06B
:1057C00096E32191222371F08093E9003093EB005E
:1057D000DF0111972C912093EC009093ED008F5FE7
:1057E000873079F78EE78093EA001092EA008F897C
:1057F000809341040FCF8B8D9C8D0E945F2A898DF1
:10580000811105C08F2D902F0E9493259BCF0E9460
:1058100003276F2D702F0E94A12694CF8093E9005B
:105820008091F200882319F08AE38093E8000895BC
:105830001F920F920FB60F9211242F933F934F9305
:105840005F936F937F938F939F93AF93BF93CF9308
:10585000EF93FF93C091E1008091E100837F8093FB
:10586000E100C3FF0FC01092E90081E08093EB00DC
:105870001092EC0082E38093ED001092410488E0E6
:105880008093F000C2FF15C083E00E940E2C80912F
:105890004304882329F0809143048150809343047A
:1058A00080914204882329F08091420481508093A2
:1058B0004204C4FF23C08091E2008E7E8160809309
:1058C000E2008091E1008F7E8093E10080913F04AF
:1058D0008E7E806180933F04FF91EF91CF91BF91C5
:1058E000AF919F918F917F916F915F914F913F9178
:1058F0002F910F900FBE0F901F901895C0FFECCF07
:105900008091E2008E7E80618093E2008091E100D0
:105910008E7E8093E10080913F048E7E8160DACF9D
:10592000109241041092400410923F040E94F72804
:10593000E1EEF0E080818E7E80838DE08093E20056
:10594000559A209A08958091E0008D7F8093E00021
:105950008091E00081FD11C080913F0480FF0DC067
:105960008091400481FF09C00E94F7288091E000E7
:1059700082608093E00081E0089580E008950895BA
:105980001092A5041092A6040895CF93DF93CDB78B
:10599000DEB769970FB6F894DEBF0FBECDBFFC012E
:1059A000DB018C918F5F8C939E012D5F3F4F8DE0CB
:1059B000D9011D928A95E9F729E0298384E08A8339
:1059C00091E09D8383E08E832A8721E22B879C8749
:1059D0009D879F8722E2288B27E02B8B25E02C8B4D
:1059E0008E8B20E430E0388F2F8B998F82818B83D0
:1059F00095858685998B8A8B838180688D8B49E11B
:105A000050E0BE016F5F7F4F80E00E946A2A699676
:105A10000FB6F894DEBF0FBECDBFDF91CF910895D2
:105A2000EF92FF920F931F93CF93DF93FB0120819F
:105A30002138A1F52381223289F5DC0112964C919F
:105A4000248135814217130649F5EC0181E00E945B
:105A5000732F0B851C85F12CE12C0115110589F0A4
:105A6000F801448155816281738180E80E946A2A2D
:105A70008F3F980761F0E80EF91ED8010D911C9137
:105A8000ECCF81E08F8780E00E94732FC701DF9108
:105A9000CF911F910F91FF90EF90089590E080E0DB
:105AA000F6CFCF93DF93EC01DB012A8114968D9121
:105AB0009C9115972817190659F411968C911197F6
:105AC0009C91913A39F4982F9D7F81E0913051F06B
:105AD00080E008C09132E1F78B3039F412968C9156
:105AE0008F8781E0DF91CF9108958A3021F413965A
:105AF0008C91888BF6CF893059F716968D919C91B1
:105B00008230910539F462E070E0CE0141960E9446
:105B1000902ADECF0197E1F661E070E0CE01429677
:105B20000E94902A198AD4CFFC01A385B4851097CE
:105B300071F47487638785859685DB0114962D91B2
:105B40003C91820F931F968785870895DC018D9184
:105B50009C9111970097D1F76D937C93ECCFAF9206
:105B6000BF92CF92DF92EF92FF920F931F93CF934A
:105B7000DF931F92CDB7DEB77C0169836A015901BB
:105B800041E050E0BE016F5F7F4FFC0183810E94C6
:105B9000B9298C0197FD0BC0F7018381A501B601DE
:105BA00080640E94B929080F191F97FD8C01C80154
:105BB0000F90DF91CF911F910F91FF90EF90DF90A9
:105BC000CF90BF90AF900895CF92DF92EF92FF9267
:105BD0001F93CF93DF93162F7A0169010E94AF2D97
:105BE000EC01E0916002F0916102309729F09C0194
:105BF000A601B701812F0995CE01DF91CF911F91A9
:105C0000FF90EF90DF90CF900895CF93DF93EC015A
:105C100081E08C838D839E01265F3F4F3F832E83DF
:105C2000198618862AE831E0398328831C861B866A
:105C30001E861D868F87888B198A1A8A81EC8A872F
:105C40000E940327BE01DF91CF910C94BF26809163
:105C5000A704811107C08FEA94E00E94052E81E01D
:105C60008093A7048FEA94E00895FC011582809147
:105C7000C804811113C01092D1041092D0048EE098
:105C800095E09093D3048093D2048AE390E09093BC
:105C9000D5048093D40481E08093C8040E94272E09
:105CA00060ED74E00C94942D0F93FC0161834283AA
:105CB000238304830F91089525E0FC0111922A9516
:105CC000E9F70895FC019081692B60830895CF93D3
:105CD000DF93EC010E94272E25E030E0AE0161E069
:105CE000DF91CF910C94E42DCF93DF93EC01988159
:105CF0008D8198130CC08981811109C08A8181111D
:105D000006C08B81811103C08C81882329F0CE01CC
:105D10000E94672E88818D83DF91CF910895CF9364
:105D2000DF93EC010E945C2ECE01DF91CF910C94A9
:105D3000742E0C948F2E82EC94E00C94352ECF931D
:105D4000DF93CDB7DEB769970FB6F894DEBF0FBE0D
:105D5000CDBFFC01DB019C919F5F9C939E012D5F59
:105D60003F4F81E1D9011D928A95E9F729E0298306
:105D700084E08A8391E09D8383E08E832A8721E2F9
:105D80002B879C879D879F8722E2288B25E3298B81
:105D900027E02B8B25E02C8B8E8B20E430E0388F96
:105DA0002F8B998F82818B83838180688D8B49E1D2
:105DB00050E0BE016F5F7F4F80E00E946A2A6996C3
:105DC0000FB6F894DEBF0FBECDBFDF91CF9108951F
:105DD0000F931F93CF93DF93EB018A01FC01838123
:105DE00080640E94B929E0916002F09161023097CD
:105DF00049F09C01A801BE0187E0DF91CF911F917E
:105E00000F910994DF91CF911F910F9108950A97F7
:105E10000C94E82EDC01FB0112962C9112978481E0
:105E200095812817190641F491818081813A31F4D6
:105E30009D7F81E0913009F080E008958132E1F7A3
:105E40009B3029F4828152968C9381E008959A3098
:105E500099F7828153968C93F8CFFB0120812138EA
:105E6000B1F42381223299F4DC0112964C911297FD
:105E7000248135814217130651F421E052962C9368
:105E800045E350E068E475E080E80C946A2A90E00D
:105E900080E00895CF93DF93EC0181E08C838D83C4
:105EA0009E012F5E3F4F3F832E83198618861D86E5
:105EB0001C861F861E86188A26E931E039832883CE
:105EC00024EA31E03B872A878A8B8B8B81EC898B94
:105ED0000E940327BE01DF91CF910C94BF2686ED6F
:105EE00094E00C944A2F0895AA1BBB1B51E107C0F4
:105EF000AA1FBB1FA617B70710F0A61BB70B881F5A
:105F0000991F5A95A9F780959095BC01CD010895E8
:105F100097FB072E16F4009407D077FD09D00E9456
:105F2000742F07FC05D03EF4909581959F4F0895FE
:105F3000709561957F4F0895A1E21A2EAA1BBB1B95
:105F4000FD010DC0AA1FBB1FEE1FFF1FA217B30745
:105F5000E407F50720F0A21BB30BE40BF50B661F5B
:105F6000771F881F991F1A9469F76095709580951F
:105F700090959B01AC01BD01CF010895EE0FFF1F6D
:105F80000590F491E02D0994A29FB001B39FC00148
:105F9000A39F700D811D1124911DB29F700D811D55
:105FA0001124911D08950E94C42FA59F900DB49FA8
:105FB000900DA49F800D911D112408950024A7FD2C
:105FC00000942A0F301D401D501D601D701D801D46
:105FD000901D08950024A7FD00942A173005400560
:105FE000500560057005800590050895FB01DC01F2
:105FF00002C005900D9241505040D8F70895FB0122
:10600000DC018D91059080190110D9F3990B089549
:10601000FB01DC014150504030F08D91059080191A
:1060200019F40020B9F7881B990B0895FB01DC01D6
:1060300004C08D910190801921F441505040C8F75F
:10604000881B990B0895FB01DC0102C001900D92A1
:1060500041505040D8F708956817790768F4FB015C
:10606000DC01E40FF51FA40FB51F02C002900E92D1
:1060700041505040D8F708950C942330F999FECF41
:1060800092BD81BDF89A992780B50895262FF99978
:10609000FECF1FBA92BD81BD20BD0FB6F894FA9A0B
:0C60A000F99A0FBE01960895F894FFCF06
:1060AC0003FFE60A01290032000140000101000152
:1060BC007F02C409FA00FFFFFFFF00000000000090
:1060CC0000000000000000000000FFC800FFFFFF00
:1060DC00FF00E100000000000000C1808100000012
:1060EC00FFFFFFFFFFFFFFFFFFFFFFFF6174726504
:1060FC00757300AF0197663534C69436F6F796374C
:10610C00009091939200000000CA0C620CAD0C5BE5
:10611C000C000000001C256825432548254B255BF9
:10612C002532250D0A0000000000512DC52C102D24
:10613C002004000000000A2F9F2E2D2F5B0CE82E50
:06614C00F6FF0000072F22
:00000001FF
